:030000000219FDE5
:03000B000200AA46
:03002B0002018748
:03005B000203336A
:0300730002032065
:1000800002030406080C10182030406080040608A3
:100090000C10182030406080A0C00003070F1F0D17
:1000A0000D0403060D0503030202C2AF306308C24C
:1000B0006385798AD2AF32C0D0C0E0206221E525C5
:1000C0006016E473E525F4C3334009758A00D263F2
:1000D000F57901D6F58AD262D0E0D0D0D2AF32C362
:1000E000E526334009758A00D263F57901F0F58A77
:1000F000C262E526F4602F30682520720DD0E0D072
:10010000D0C293C297C294D2AF32C293C297C29464
:10011000206F0C2065097406D5E0FDE57B4290D088
:10012000E0D0D0D2AF32758A00D263757900C28D2B
:10013000D262211F01C4306805206502D29301C438
:10014000306805206502D29401C43068052065023C
:10015000D29701C4C29230680A2065077406D5E0C0
:10016000FDD29301C4C29530680A2065077406D594
:10017000E0FDD29401C4C29630680A206507740677
:10018000D5E0FDD29701C4C2AFC2AD53E6EFC0D0F7
:10019000C0E0D2D3D2AFE57A6009E5776005757724
:1001A000004123757701C2CEE52A60072074491506
:1001B0002A21F87800790020742EE580307E01F441
:1001C00030E50278FF53DACF207E0343DA20307E19
:1001D0000343DA10C2D8C271E580307E01F430E505
:1001E0000279FFC3E89970CB306103752A4020740F
:1001F00003752A40885CD27020740DE52B600415CD
:100200002B410843DA01C2D8207002411BA85C20B0
:100210006102C270207402411988227882B60403F8
:1002200085222420CF0AD0E0D0D043E610D2AD32D0
:10023000C2CF053AE57A6009E57860057578006116
:10024000167578017802E52A6005307402152AC314
:10025000E55C94014005755F00416C75600075694F
:1002600000E55F2401F55F5003755FFF7982B702F7
:100270000D306E1DC3E52294324016854C227982E2
:10028000B7030E306E0BC3E52294324004798E879B
:1002900022C3E523952260084004152341A00523CD
:1002A000D8CA0569E56970021569D56A69756A0178
:1002B0007808E56B60497805C3E569956B4057C3DD
:1002C000E569956C50087801756A030202DAC3E5A6
:1002D00069956D50057801756A01C3E56295244002
:1002E0001E7982B70402610B206E14852462E569D1
:1002F000046003856B69756A0175233C020316E58A
:10030000622850057562FF610BF562E562047006B4
:100310007560FF7569FFD0E0D0D043E610D2AD32F2
:10032000C2AF53E67F7592FA7593FFC26075910470
:10033000D2AF32C2AF53E6EFC2ADC0D0C0E0C0F022
:10034000D2D3D2AFA8FBA9FCE57A6007C3E913F9C1
:10035000E813F8C2D830710261A553DACF207E03CA
:1003600043DA10307E0343DA20D271E580307E011B
:10037000F420E502617C88278928A18A53DACF20FE
:100380007E0343DA20307E0343DA10C2D8C27130D4
:100390007402A1767800E580307E01F430E502A198
:1003A00076885CA15E53DACF207E0343DA20307E6C
:1003B0000343DA10C271206102817E53DACF207EBE
:1003C0000343DA10307E0343DA20C2D8D271885753
:1003D0008958C3E89555F8E99556F97B007E087A67
:1003E00000C3E8948CE994005005755B0081708827
:1003F0002178A2E6A8216055C3E894C8E99400508A
:1004000008E4D2E4FB7A0A814BC3E89468E99401DA
:100410005008E4D2E3FB7A0F814BC3E894D0E9940F
:10042000025008E4D2E2FB7A1E814BC3E894A0E9B3
:1004300094055008E4D2E1FB7A3C814BC3E89498E0
:10044000E994085008E4D2E0FB7A787E00C3E8958E
:1004500059FCE9955AFD30E70AECF42401FCEDF46F
:100460003400FD755B00C3EC9AED9E5003755B0193
:0F0470008859895A8557558558567802A15EC319
:10047F00E89527F8E99528F9307C02A142307B02F4
:10048F00A142307A02A13B20750281A1E9FDE8FC6F
:10049F0081C0E9C313F9E813F8307902A13BE9C32E
:1004AF0013F9E813F8307802A13BE9C313FDE81301
:1004BF00FC20612CC3EC941CED9402400281D7ED1B
:1004CF00701EC3EC94C850180529E5297002152930
:1004DF00C3E529940A5002A176755C00D270A1760B
:1004EF00E529600215297400207F037896E624FA27
:1004FF00FEE43400FFC3EC9EFCED9FFD5006780038
:10050F007900A142C3EC94FFED9400400678FF7987
:10051F0000A142EC8572F0A4C5F0A2F733F8790080
:10052F00400302055E78FF790002055EE9C313F907
:10053F00E813F8307C0EE9600278FFC3E81338F84F
:10054F00E43400F9C3E894FFE99400400278FF888F
:10055F005CD270206102A176741FF4552F4BF52FDA
:10056F00C274EB7002D274752A40307403752A0A74
:10057F00306102A18A20740353DAFE207403752BB5
:10058F0020D0F0D0E0D0D0D2AD43E61032790102C6
:10059F0005BA79030205BA790A0205BA791E02056E
:1005AF00BA79640205BA79C80205BA7817E4D5E0BA
:1005BF00FDD8FAD9F6227A147B780205E17A107BFE
:1005CF008C0205E17A0D7BB40205E17A0B7BC80240
:1005DF0005E1E573D5E001227902E4C295D5E0FD8E
:1005EF00D294D5E0FDC294D5E0FDD295D5E0FDE9DA
:1005FF0020E002D29330E002D297E573D5E0FDE917
:10060F0020E002C29330E002C2977496D5E0FDD984
:10061F00C9EAF8D5E0FDD8FBDBB8C29522C37C0050
:10062F007D0075F00005F0EA33FAEB33FB50F6EB83
:10063F0013FBEA13FAC3E9FFE8FEE89AF8E99BF91E
:10064F005004EFF9EEF8B3EC33FCED33FDD5F0DFEA
:10065F00EDF9ECF822E889F08A20D2D4F8A9F07BE2
:10066F000030F70B7BFFF42401F8E9F43400F9E8CC
:10067F008520F0A4ADF0F8E98520F0A4AFF0FEEDF1
:10068F002EF974003FFA7C04C3EA13FAE913F9E870
:10069F0013F8DCF48BF030F70AE8F42401F8E9F4EE
:1006AF003400F9E889F0C2D4F8A9F0227882B604B0
:1006BF000302075AC3E55C9419401EE52D540670DA
:1006CF0018206E3678057994E7146007780A14605D
:1006DF00027812C3E54198401F306E098564627538
:1006EF0069FF756A01852224E4F544F545F546F561
:1006FF0047F548C26E02075AD26E7994E714701309
:10070F00E523F43333F913F8E9540104F9E854FEFF
:10071F0002074EE714147014E523F4333333F9133F
:10072F00F8E9540304F9E854FC020756E523F433BF
:10073F00333333F913F8E954070404F9E854F8C3D1
:10074F009440F8E99400F98844894522C3E54113A0
:10075F00F9E54013F8C3E54498F8E54599F9500CCD
:10076F00C3E89480E994FF4016020792C3E8947F90
:10077F00E994005003020792787F7900020792787C
:10078F008079FF8849894A22E5492546F8E54A35A7
:10079F0047F9854A20E4300701F43548FA30E70974
:1007AF00C3EA94F040150207D0C3EA940F50030236
:1007BF0007D078FF79FF7A0F0207D0780079007A97
:1007CF00F0C3E5249561500AC374019524500B02C0
:1007DF0007EEE54A20E70E0207EEE54A30E7068806
:1007EF004689478A482278A5E6FAC3E54933F8E5F2
:1007FF004A33F9120664E930E70BC3E89480E994B1
:10080F00FF40130129C3E8947FE9940050020129A6
:10081F00787F79000129788079FFE820E715C3E513
:10082F002398F84009C3E894014003020850780167
:10083F00020850E8F424012523F8400302085078F9
:10084F00FF884B2278A6E6FAA847A948120664E962
:10085F0030E70CC3E89401E994FF4016020885C302
:0F086F00E894FFE99400500302088578FF7900B0
:10087E00020885780179FFE920E715C3E54B98F862
:10088E004009C3E8940140030208AC78010208ACA9
:10089E00E8F42401254BF840030208AC78FF8824C5
:1008AE002278FF20692879A1E76023E541601F7453
:1008BE00FF8541F0848539F0306A0375F005A4F8A0
:1008CE00C5F0600278FFC3E895645002A86488639F
:1008DE0022C3E54094C8E5419400E563500314013A
:1008EE00F0046002F563227883E6F520120F8B7513
:1008FE00E89012059C75E89030EDFDA8BDA9BE12DA
:10090E001031756E00756F00C3740013FD740060B6
:10091E006613FC74002CFC74003DFDECFAEDFBC379
:10092E00E89AE99B4014E56E2400F56EE56F3400FD
:10093E00F56FEA2CFAEB3DFB80E5AE6EAF6FC3E5CB
:10094E006F13F9E56E13F8C3E913F9E813F87A0398
:10095E00C3E913F9E813F8DAF7AA201A7009756ECD
:10096E0000756F000209851AEA6008EE28FEEF395D
:10097E00FFDAF88E6E8F6F2275E890227883E6FF8D
:10098E0030EDF9A8BDA9BE0570C3E57094084052BC
:10099E00757000E9FA79A0E76044EA7007E57160C6
:1009AE001B0209BEC3E895716010E5715006600C1C
:1009BE00140209CA0460F90209CAE571F571C394FB
:1009CE0072401B7561C0C394044013756180C3945B
:1009DE0004400B756140C39404400375610075BB00
:1009EE000922EFC39401601F7400601BC3E894FFDB
:1009FE00E994035012C3E8956EE9956F5009E561CD
:100A0E00600C1561020A1CE561F460020561A861C3
:100A1E00C3E524985002A824C3E89562400AA86250
:100A2E00E562F4600385626188258826E570B40767
:100A3E000375BB1022743279A787F0A4C5F0A2F714
:100A4E0033F8C3E895614002A8618822882488257E
:100A5E0088268864227540007541F022C2AF75C8A1
:100A6E0020A8CCA9CDAA3A30CF010A75C824D2AF9E
:100A7E00C3EA13FAE913F9E813F8AB3BAC3C883B35
:100A8E00893CC3E89BF8E99C20690A547FF93066DB
:100A9E0002618741E1AD3D8A3DF9EA9D547FFA60DE
:100AAE000478FF79FFAE3EAF3F8B3E8C3FA83BA94B
:100ABE003CC3E89EF8E99FF9C3E54113FBE54013FB
:100ACE00FAE82AF540E93BF54150067540FF7541BD
:100ADE00FF612EAA40AB41AC40AD417E047F02C304
:100AEE00EB9404400D1E1FC3EB94084005206A02D0
:100AFE001E1FC3ED13FDEC13FCDEF7C3EA9CFAEBED
:100B0E009DFBEF6009C3E913F9E813F8DFF7EA2854
:100B1E00FAEB39FB8A408B4150067BFF8B408B41B1
:100B2E00C3EB94025002D2663069047F0361597898
:100B3E0092E6FFC3E537948240110FC3E53794A0C8
:100B4E0040010FC3EF940640027F057E02E541C4CB
:100B5E00540FF9E541C454F0F8E540C4540F28F899
:100B6E00C3E89EFAE99400FB4009C3EA9402EB94B1
:100B7E000050047A02E4FB61D3AA40AB41EBC4FE01
:100B8E00EAC4540F4EFCC3EA9CFAEB9400FBC3E894
:100B9E0013C313F8EA28FAEB3400FB8A408B41C3E7
:100BAE00EB94024002C2667802EBC4FE7B00EAC4FC
:100BBE00540F4EFAC3EA98FA4005C3940250027AD3
:100BCE00027892E6FF30600261D38551928552938E
:100BDE00D26043E680C3E49AF8E49BF9C3E833F8A5
:100BEE00E933F93066028166E8FAE9FBD3E913FDD1
:100BFE00E813FC88518952C3EF94036038EF20E06C
:100C0E000DE82CF8E93DF9ECFAEDFB020C2FE82883
:100C1E00F8E939F9C3E82402F8E93400F97AFE7BE1
:100C2E00FFC3EF9403400E8A538B54884D894E8C2C
:100C3E004F8D50819A885389548A4D8B4E8C4F8D8F
:100C4E00503069127553F07554FF754FF07550FFA3
:100C5E007551F07552FF819AE8FAD3E813FC88516A
:0F0C6E00C3EF94036020EF20E007E82CF8ECFAC6
:100C7D008186E8282402F87AFEC3EF940340088A9F
:100C8D0053884D8C4F819A88538A4D8C4FE568C39C
:100C9D00335002646BF56830600281A4753402D262
:100CAD006043E680E52D5406602DA840A941C3E9B7
:100CBD0013F9E813F8306904E92440F9C2AF53E69B
:100CCD007F759100C3E498F594E499F595759104B9
:100CDD00D26043E680D2AF22D26475430075200006
:100CED00306C03752040020D04D2647543007520ED
:100CFD0040306C0375200078017901206620E52DC8
:100D0D0054066002C2647914E541C313700104F8FE
:100D1D00C3941440027814306904781B791BC3E81E
:100D2D0033F8C3E933F9206010E543600C306903F3
:100D3D00D53404D26DA1BB91AC0543E59BF4544071
:100D4D00B52002A1A530690908C3E899400118A191
:100D5D003320640A08C3E8994002A104A133C26498
:100D6D00C2AF53E67F75910030661275940075958C
:100D7D00F0759104D26043E680D2AFA104E5417EC7
:100D8D00FFC3334009C3334005C3334001FEC3E401
:100D9D009E759400F595A17EC3E53394015002A193
:100DAD0004306402A104D802A1B9A133C26DC2AF4F
:100DBD0053E67F75910085539485549575910485FF
:100DCD004D92854E93D26043E680D2AFE52D540609
:100DDD006008206A020533020DF7306D0D206C0A94
:100DED00206407158115810216A82278003064024F
:100DFD007801E53775F007A4F9E5F028F5F0E9A2DB
:100E0D00F013A2F113A2F213F537C39478500375C2
:100E1D003778C3E53795384008D265C293C297C27B
:100E2D0094306002C12E854F92855093D26043E677
:100E3D008022207D16C2AF754202C295D2923062D9
:100E4D0002D297D2AF759F8002102EC2AF754202AB
:100E5D00C295D296306202D293D2AF759F800210A6
:100E6D002E307243207D20C2AF754203900165750F
:100E7D007B20C297C296306204D294C18CD295D297
:100E8D00AF759F8902102EC2AF7542039001657533
:100E9D007B20C293C292306204D294C1ACD295D25F
:100EAD00AF759F8102102E207D17C2AF7542039042
:100EBD000140C297306202D294D2AF759F89021061
:100ECD002EC2AF754203900140C293306202D2949C
:100EDD00D2AF759F8102102E207D16C2AF754204D0
:100EED00C292D296306202D294D2AF759F81021017
:100EFD002EC2AF754204C296D292306202D294D203
:100F0D00AF759F8902102E307243207D20C2AF75C0
:100F1D004205900154757B04C294C295306204D28F
:100F2D0093E132D292D2AF759F8002102EC2AF756F
:100F3D004205900176757B40C294C295306204D211
:100F4D0097E152D296D2AF759F8002102E207D1759
:100F5D00C2AF754205900136C294306202D293D26F
:100F6D00AF759F8002102EC2AF75420590014AC227
:100F7D00943062EBD297D2AF759F8002102E207DF8
:100F8D0016C2AF754206C296D295306202D293D286
:100F9D00AF759F8902102EC2AF754206C292D295CF
:100FAD00306202D297D2AF759F8102102E307243FC
:100FBD00207D20C2AF754201900176757B40C293B2
:100FCD00C292306204D297E1D8D296D2AF759F818A
:100FDD0002102EC2AF754201900154757B04C29769
:100FED00C296306204D293E1F8D292D2AF759F8946
:100FFD0002102E207D17C2AF75420190014AC29397
:10100D00306202D297D2AF759F8102102EC2AF759A
:10101D004201900136C297306202D293D2AF759FD2
:10102D0089C26522900134757B00C293C297C29428
:10103D00C292C296C295C262227880760708760760
:10104D000876010876040876FF0876FF0876090809
:10105D007602087601087601788C7601087600080C
:0F106D0076B40876FF0876FF0876FF087603084A
:10107C0076FF0876010876FF0876250876D0087684
:10108C00780876C80876040876FF0876010876009A
:10109C0008767A08760A0876010876010876000840
:1010AC0076FF087600227887E6FFC272BF0302D271
:1010BC00727888C27DE630E102D27DC27E7889E604
:1010CC0030E102D27EC3EF94026008758E01D273B8
:1010DC000210E4758E00C273227880E614900080B2
:1010EC009378A5F67881E6149000809378A6F6782C
:1010FC0086E61490008D9378A7F6789FE6F8700535
:10110C00756B00212BC3E8941140027811E8282854
:10111C00F56B256B256B28F56C256B2828F56D7800
:10112C0086E6F539C394025003753902789CE6754E
:10113C0038FFB402037538A0B4030375388278A362
:10114C00E61490009A93F566113122227896E6FA0D
:10115C007897E6FB7888E6B40305C3EB940EFB3076
:10116C007F047A007BFFC3EB9AFCC3948250027C11
:10117C00827572000572EC8572F0A4C3E5F0947D63
:10118C0040F222D27F31581205AB1205AB7A007BAC
:10119C00007C101205A1E55C2AFA74003BFBDCF321
:1011AC007C04C3EB13FBEA13FADCF7FEC27F315865
:1011BC0022757C00757D00E5EF20E60375200005A7
:1011CC0020903FFFE520146006901FFF14600093F1
:1011DC0004600375EF1653D9BF7581C043FF8012AD
:1011EC00059C75EF0643B203E5B3240220E70DF529
:1011FC0021E5E320E0068521B343E301113175803D
:10120C00FF75A40075F1F075D4DF75900275A5FC1F
:10121C0075F2FD75D50275A61075A0FF75F3F17505
:10122C00E2411131E4F8F6D8FD7568011146121748
:10123C000678988673753001C2AF1205B51205C5D4
:10124C001205AB1205CC1205AB1205D31205AB126D
:10125C00182C1205B51205B51205B0C2AF757C007D
:10126C00757D0078FA79FA308507D9FBD8F7021C1E
:10127C000011B211E53157315878988673113175D8
:10128C00A90075B680757A0075881075890275C8C5
:10129C002475910475D84075A82275B80275E6902E
:1012AC00759B80759D0075D10E75BCC075BB09759D
:1012BC00BA1175E88012059CD2AF1208F57536008C
:1012CC0053DACF207E0343DA20307E0343DA104317
:1012DC00DA01C2D8C2711205B5D2617B037A0CE572
:1012EC005B70077A0CDB030212671205AB207003EC
:1012FC00021267C270E55CC3940240E1E52F541FF3
:10130C00855E5DF55EB55DD5DAD5C26153DACF2069
:10131C007E0343DA20307E0343DA10C2D8C27178E0
:10132C00A2E67008D274E52F54E0F52FC27575292A
:10133C00001205B0307409C3E529940A4002D27535
:10134C001205A178023074027800C3E55C9840F075
:10135C00C2AF1205C51205C51205C5D2AF1205B52F
:10136C00754C001205A1788CE6C39401500302144D
:10137C005CE530C39401500302145C757CA5757D4B
:10138C00F1207435C3E55C94FF500302145CC2AFCA
:10139C001205DAD2AF1205B0C3E55C940150EFC26E
:1013AC00AF1205C51205A61205C5D2AF1205B0C302
:1013BC00E55C94FF40E90218B17F05D27F315812E9
:1013CC0005B0C2AFC27F3158AE5CC3E55C947FD22E
:1013DC00AF5002816C12059CC2AF1205DAD2AFDF9E
:1013EC00DA318FC3EE94057897F61205B5121834DE
:1013FC007F0AD27F31581205B0C2AFC27F3158AECE
:10140C005CC3E55C947FD2AF50E612059CC2AF1270
:10141C0005C51205A61205C5D2AFDFD6318FEE2455
:10142C00037896F6F87997E7C394824003985006B0
:10143C00E824827897F61205B51217471218631232
:10144C0005B03158C3E55C94FF500261870218B1B6
:10145C00757C00757D00C3E55C954C4003855C4C48
:0E146C001205B078017988E7B403027805C351
:10147A00E55C984002616FC2AF1205DA1205DA1212
:10148A0005DAD2AF1205B5753000E4F531F532054B
:10149A0031E531F4703E0532789AE6781914601213
:1014AA00783214600D787D14600878FA1460037538
:1014BA003200C3E53298401C113112059C15327571
:1014CA00310078998673C2AF1205DAD2AF7898865E
:1014DA00731205B01205A6E52A7005307402416739
:1014EA0078012074027806C3E55C9840A21205B020
:1014FA00E52A7003021267C2AF1131E4F522F5231F
:10150A00F524F525F526F567D2AF7885E6C333F5D8
:10151A0065E4F544F545F546F547F548F570F52CCB
:10152A00F52DF53775700875BB1012059C120986E2
:10153A0030EDFDA8BDA9BEE97001F8887112098ACB
:10154A0075700875BB1011B2C2AF7561FF120A43FC
:10155A00852261852262852263D2AF7522017524B4
:10156A0001752501752601856069756A0175B69050
:10157A0075A903757A017888E6B40307C27D3076C7
:10158A0002D27DD268D269753300120F8B120FBA5C
:10159A00120A63120A6A120A63120A6A120A6312A6
:1015AA000CF61206BB120DF8120E3F120A6A120C42
:1015BA00E5306E0312075B2066031208AF3066033C
:1015CA001208DF120DF8120E6E120A6A120CF630A9
:1015DA006E03120797120DF8120EE5120A6A120C20
:1015EA00E5306E031207F5120DF8120F14120A6A8B
:1015FA00120CF6306E03120853120DF8120F8B12EA
:10160A000A6A120986120CE5120DF8120FBA1209AB
:10161A008A120A6A30692C85646185646285606908
:10162A00756A0179187A0CC3E533994009C269D2FF
:10163A006A8A3502164DC3E55C940140030215A976
:10164A000216B0306A1D206C1AE535147006C26A9B
:10165A00D26BA1A9F535C3E55C940140030215A933
:10166A000216B0753600C3E55F94014009856462CD
:10167A00856069756A0178FA79A4E760027803C31C
:10168A00E55F985021307404E52A601A78F0306CCE
:10169A00058564617820C3E541985002A1A9053601
:1016AA00E55C6002C1B3753600C2AF11317887E6D6
:1016BA00FE760211B27887EEF6E4F522F523F524D8
:1016CA00F525F526F565752C00752D0075A90075AB
:1016DA00B680757A00D2AF1205B0113178A4E660EF
:1016EA0006D292D295D296307406E52A70024167E4
:1016FA00788DE6C394014002614C8194901A0D786A
:10170A0020121789E520B4A50CA3121789E520B485
:10171A005A030217271146121747021746901A034F
:10172A0078807B0A121789A308DBF9901A0F788C44
:10173A007B19121789A308DBF9901A2822C2AF1263
:10174A0017CC1217A9901A00740E12178EA37407D9
:10175A0012178EA3741512178E901A0378807B0ABB
:10176A0012178DA308DBF9901A0F788C7B191217C0
:10177A008DA308DBF91217DF1217BD901A2822E48D
:10178A0093F622E6438F01538FFDFFC3E583941C32
:10179A00400122EF857CB7857DB7F0538FFE224347
:1017AA008F02438F01857CB7857DB7901A0DF05360
:1017BA008FFC22901A0D74A5F18E901A0E745AF1AC
:1017CA008E227A3079D07820901A40F189E520F774
:1017DA0009A3DAF7227A3079D0901A40E7F18E0914
:1017EA00A3DAF922AB74A875BB01027980BB0202A5
:1017FA007981BB03027982BB04027994BB05027921
:10180A0083BB06027986BB07027992BB08027987F5
:10181A00BB0902799CBB0A027988BB0B027989E869
:10182A00F7227C051205B5DCFB22C2AF1205C512F0
:10183A0005CC1205D31205DA1205A61205C5120542
:10184A00CC1205D31205DA1205A61205C51205CC6B
:10185A001205D31205DAD2AF22C2AF1205DA120587
:0D186A00D31205CC1205C51205A61205DA31
:101877001205D31205CC1205C51205A61205DA12F8
:1018870005D31205CC1205C5D2AF22AE74AF75C20F
:10189700AF1205C51205C51205C51205A6DEF2125F
:1018A70005DA1205A6DFF8D2AF221134112C112C5C
:1018B70075740175750175760011927C05AD5C1222
:1018C70005B5C3ED955C70F5C3E55C9401400AC3AB
:1018D700E55C94FF40340218EF1217EE1217471118
:1018E70034C2AF75EF16112CDCD30576C3E57694B9
:1018F70003500280C4112C0575E5741490009F9362
:10190700F808C3E57598500280AC112C112C0574AA
:10191700C3E574940C5002809A121046121747C2FE
:06192700AF75EF16112C54
:0319FD000211BD17
:101A00000E071507070104FFFF09020101A55A018E
:101A100000B4FFFFFF03FF01FF25D078C804FF01DA
:091A200000FF0A010100FF00FFB4
:101A4000234656544C69626565333041232020207B
:101A500023424C48454C492346333930232020202B
:101A60002020202020202020202020202020202076
:101C0000C2AFC2D353D9BF7581C043B20343FF8073
:101C1000752438752503B1DC7529A5752AF175E29F
:101C20004043F12053A4DF75D4FFD2857DFA7803B9
:101C300079E67C10752200752300901DE97B0675FE
:101C400024987525013085028145208508D8FBD967
:101C5000F9DCF781B7308508D8FBD9F9DCF781B713
:101C6000B19CE493A3C39A6004DDC381B7DBDBB10D
:101C70008E6002812E7B08E493FAA3B16FDBF87AC1
:101C800030B16F752200752300B18EEAFCEBFDC305
:101C9000ED94FE400EB18E8A278B28ED30E0048A49
:101CA000828B83B18E7AC270D8C3ED94FE601950D6
:101CB000CEBD002BEC600F7520007521FF7529004B
:101CC000752A000200008100A827A9280809D80465
:101CD000D90281DCB192EA89AAF281CE0D81A3C337
:101CE000ED94035053EDA2E092007AC5C3E58294CF
:101CF00000E583941C508A200010438F02438F011B
:101D00008529B7852AB7F0300029A827A92808090E
:101D1000438F01538FFDD804D902A133C3E58394C7
:101D20001C4003A3A11689AAE28529B7852AB7F02A
:101D3000A3A116538FFC817F7AC1BD030CE493A34A
:101D4000FAB153DCF8B14B817F8181AA22AB23B178
:101D50006FEBFAEA6222752608C3E52313F523E543
:101D60002213F52250066323A0632201D526EAB18F
:101D7000DCB1DC75260AEAF4200102D285300102CA
:101D8000C285B1DCC3134002C201D526EB22B19259
:101D9000EAFB208502A192308502A197752608AE44
:101DA00024AF25C3EF13FFEE13FEB1E0B1DCC3EAAD
:101DB000133085024480FA30E703632201C3E52330
:101DC00013F523E52213F52250066323A0632201B5
:101DD000D526D9E52265236523F52222AE24AF2539
:101DE0000E0FDEFEDFFCD20122424C48656C6934E6
:071DF000373163F390060197
:00000001FF
